:03000000022F1FAD
:0C2F1F0078FFE4F6D8FD75814A022F66A9
:100EB10020000A3C2E2E2E3E004950436F6E6E6577
:100EC10063745245510A004950436F6E6E656374F5
:100ED100000A49504E6F41434B210A003E432C56B4
:100EE1002C43432CC0E4E0EFF2E5F020D1E8EDEA39
:100EF100EEEC49500A003E432C4D41432C25303243
:100F010062583A25303262583A25303262583A25D1
:100F1100303262583A25303262583A2530326258BE
:100F21002C4D414320E0E4F0E5F10A003E432C560C
:100F310045522C20332E3220EEF2202573202573CA
:100F41002CC2E5F0F1E8FF20495020ECEEE4F3EB90
:100F5100FF0A004D617920303520323030380031C0
:100F6100323A33343A3537003E432C4C442C5052FC
:100F71004F473A2020202020202020202020202000
:100F81002020202020202020202020202020202060
:100F91002020202020202020202020202020202050
:100FA1002020202020202020202020202020202040
:100FB10020202020202020202CC4E0F2E020EFF08F
:100FC100EEF8E8E2EAE828F4E0E9EB290A003E2A33
:100FD1002C312CCEF1EDEEE2EDFBE520EFE0F0E07F
:100FE100ECE5F2F0FB20F1E5F2E5E2EEE3EE20E8DC
:100FF100EDF2E5F0F4E5E9F1E00A003E412C413083
:10100100312C2562752E2562752E2562752E25627D
:10101100752C495020E0E4F0E5F120E0E4E0EFF246
:10102100E5F0E00A003E412C4130322C2562752E5C
:101031002562752E2562752E2562752C495020E09A
:10104100E4F0E5F120EEF1ED2E20F1E5F0E2E5F03E
:10105100E00A003E412C4130332C2562752E256279
:10106100752E2562752E2562752C495020E0E4F01D
:10107100E5F120F0E5E72E20F1E5F0E2E5F0E00A08
:10108100003E412C4130342C2562752E2562752E8F
:101091002562752E2562752CCCE0F1EAE020F1E5A0
:1010A100F2E80A003E412C4130352C2562752E258F
:1010B10062752E2562752E2562752CD8EBFEE70A26
:1010C100003E2A2C312CC4EEEF2E20EFE0F0E0ECB4
:1010D100E5F2F0FB20F1E5F2E5E2EEE3EE20E8EDEA
:1010E100F2E5F0F4E5E9F1E00A003E422C5330313B
:1010F1002C2562752CC6E4E0F2FC20E7E0EFF0EE6F
:10110100F1E020F1EEE5E4E8EDE5EDE8FF20EEF2B7
:1011110020F1E5F0E2E5F0E00A003E422C533032E6
:101121002C2562752CCEE1ECE5ED20F120F1E5F006
:10113100E2E5F0EEEC20E1E5E720EAE2E8F2E0EDBD
:10114100F6E8E90A003E422C5330332C2562752C17
:10115100CFE5F0E5E7E0EFF3F1EA20EFF0E820EF8B
:10116100EEF2E5F0E520F1E2FFE7E820F120F1E51C
:10117100F0E2E5F0EEEC0A003E454E440A000A4476
:10118100756D7058202020202030302030312030E3
:101191003220303320303420303520303620303783
:1011A1002030382030392030412030422030432057
:1011B1003044203045203046000A3A003A20000AE7
:1011C100000A44756D7044202020202030302030EA
:1011D1003120303220303320303420303520303649
:1011E1002030372030382030392030412030422023
:1011F1003043203044203045203046004572722073
:101201006B657900526420656570726F6D0A0052DA
:1012110064204D454D0A00526420436F64650A0005
:10122100577269746520436F64650A00446562758D
:10123100674950204F4E0A00446562756749502046
:101241004F46460A00446562756755736572204FC3
:101251006E0A00446562756755736572204F464694
:101261000A0044656275674D7367204F6E0A00443A
:10127100656275674D7367204F46460A00436F6E7E
:10128100666967206C6F636B210A00577220656580
:1012910070726F6D0A00205361766520656570720A
:1012A1006F6D210A00457272204D414321004C6F40
:1012B10061643E3E002A003C4130313D003C4130FA
:1012C100323D003C4130333D003C4130343D003C37
:1012D1004130353D003C21003C5330313D003C5311
:1012E10030323D003C5330333D003C5330353D00FE
:0612F1003C5330363D00C5
:0637A6000147000145008F
:1037ED00C28E438910758BFF758DB7D2ABD28E22E9
:03001B00022E8F23
:102E8F00C0E0C083C082C0D0C28E758BFF758DB776
:102E9F0020060675A61E75A6E10545D202E5476018
:102EAF00020547E546D3940140021546054AE54A17
:102EBF00540F7048D20EE54A543F7012D2009066FC
:102ECF008BE0600A04F0E0D394B44002D20690661F
:102EDF0086E0600204F0906104E0600214F09066F6
:102EEF008CE0D394014003E014F03005020548E56F
:102EFF0049D394644004D20680020549E544D39433
:102F0F000140021544D28ED0D0D082D083D0E0328F
:10085300C2AFC291C290D2B5C20B7D027C007F07AA
:100863001237898F25E525646060097D017F601259
:100873003724D20BE4FDFC7F0B1237898F25E52546
:1008830030E6097D04E4FF123748D20B7D017C007A
:100893007F071237898F25E5257008FD7FFF123703
:1008A30024D20B300B03126000C288C2A8C2AA75FF
:1008B300890012324790633EE0B4FA06A3E064CEA7
:1008C300607BE4F52574362525F582E43463F583EE
:1008D300E4F00525E525B443EC90633E74FAF0A3F8
:1008E30074CEF0A374CCF0906344740AF0E4A3F0E4
:1008F300A304F0A3F090633A74FFF0A3F0A3F0E431
:10090300A3F0906355740AF0E4F525E5252401FF6F
:10091300E433FE74362525F582E43463F583E0FD84
:100923001237000525E525C3944340DFE4F5A77599
:10093300A61E75A6E1907FF0F0A3F080FE906349B8
:100943007403F0A374CCF0E4906348F0122AE3C27A
:10095300B5123341C2061235CCD20BC20DC20C9074
:1009630065767408F09062B47424F0E4A3F09063A5
:100973003EE09062B6F090633FE09062B7F0906320
:1009830040E09062B8F0906341E09062B9F0906308
:1009930042E09062BAF0906343E09062BBF0754628
:1009A30001E4906577F0C207C208C209C20A200BAE
:1009B30018AF25FE7D03122926E4FF122DDF7E0EDC
:1009C3007FB1E4FBFDFC12237190668BE06003743E
:1009D30001F0E4906104F0F548906575F0F5491273
:1009E30037ED75A70775A61E75A6E1D2AFE4F549E5
:1009F300906104E0700312266C90668CE0B40111E0
:100A03009080007410F0E490668CF0D20BC20CC29C
:100A13000D908008E0F52530E405D2077410F0E569
:100A23002530E508D2099080087420F0E52530E6EA
:100A330008D2089080087440F0E548C39403401935
:100A4300908002E4F0908001F0908000F0E54894FB
:100A5300064006E4F5481235CC9080A0E0700312FE
:100A630033BC9080B8E070031234369080D0E070CD
:100A730003123570908000E0701330071012247851
:100A8300906331EFF0D3940040031200269080026C
:100A9300E07006908000E06005D2050209F0C2050F
:100AA300E4F548906104E060030209F0200B129022
:100AB3006578E0600C7E0E7FB3122759E490657869
:100AC300F030091212220B906331EFF0D3940040FF
:100AD30005E0FF12380F200803020C59121F08907B
:100AE3006331EFF070030209F0906375E054BF24A3
:100AF3007F7003020BC2147003020B9A240260037B
:100B0300020BFB200B077E0E7FBA122759200F031F
:100B1300020C5990634DE07006906351E06067905A
:100B23006682E0FF90634DE0B50724906683E0FEA4
:100B330090634EE0B50618906684E0FE90634FE044
:100B4300B5060C906685E0FE906350E06E603790CA
:100B53006351E06F6003020C59906683E0FF90637A
:100B630052E06F6003020C59906684E0FF90635378
:100B7300E06F6003020C59906685E0FF906354E0D8
:100B83006F6003020C59C2039065777401F0123849
:100B930010754601020C5990668BE060037401F0F6
:100BA30090667AE0FF906377E06F6003020C5990E0
:100BB300667AE004F0E4F546906575F0020C59306E
:100BC3000303020C59906344E070030209F090633D
:100BD30055740AF0123807D203E4F546906575F0B0
:100BE30090668604F0E4906679F0A3F0200B677EAC
:100BF3000E7FC8122759805E90668BE060037401F4
:100C0300F0300352906375E020E74B906377E0FF89
:100C1300906679E0FE6F600D906681E07007EE14D8
:100C23006F70338013906679E004F0906331E0FFD6
:100C3300D3940440031232C59060007482F0A3740D
:100C430001F0906377E0906002F07E607F007D03A7
:100C53001230320209F0200303020D71E546706879
:100C63001237FDEF60237E647F75906476E0240481
:100C7300FD123032906681E07009906355E0F546CD
:100C83000209F0E4F5460209F0906686E0D3943C4D
:100C93004036906681E0703090668604F0122D2A0B
:100CA300E4906475F0A37412F090667AE090647730
:100CB300F0A374FDF090610563A20190647963A2CF
:100CC300017F12121C56809E1237DC8F25E525B456
:100CD30001159060007483F0E4A3F07E607F007DD3
:100CE300021230320209F0E525D39401401C9060D2
:100CF300007483F0A37401F0E52524FEA3F07E6065
:100D03007F007D031230320209F0E546640160037F
:100D13000209F0906575E004F0200B077E0E7FD288
:100D2300122759906355E0C394C85004E02432F06D
:100D3300906575E0C39405400DC203E4906577F0B8
:100D43001238100209F07C667D82906349E0FAA3B1
:100D5300E0FB7F021231C37E647F75906476E024EA
:100D630004FD123032906355E0F5460209F0E54682
:100D7300640160030209F0906577E014604624FE85
:100D83006042147003020E64240460030209F0E459
:100D9300F548200F139065777404F0906575E0545F
:100DA30001F07546010209F09080027410F0E4909E
:100DB3006577F090657504F07546FA90668274FF66
:100DC300F00209F0906682E07003020E4E906475A3
:100DD3007480F09064777401F0E4A3F0A304F0A3AB
:100DE3007430F0A3747BF0E4F525747C2525F5823B
:100DF300E43464F583747DF0747D2525F582E43451
:100E030064F583E4F0E5252407906476F07C667D41
:100E130082906349E0FAA3E0FB7F021231C37E6450
:100E23007F75E5252409FD123032906681E0601B51
:100E3300123807D203E4F546906575F09066860490
:100E4300F0E4906679F0A3F00209F0300F07E49024
:100E53006577F080069065777404F07546FA0209A9
:100E6300F09080027410F0754605906575E064019A
:100E7300FFF09065777401F0EF7019906351E060B3
:100E830013FCA3E0FDA3E0FEA3E0FF90668212172C
:100E9300E40209F090634DE0FCA3E0FDA3E0FEA3B0
:0D0EA300E0FF9066821217E40209F080FE65
:010EB000221F
:10002600906376E0B444047F0180027F009063759C
:10003600E0B447047E0180027E00EE5F604A906372
:100046003EE0906377F090633FE0906378F09063D2
:1000560040E0906379F0906341E090637AF09063BA
:1000660042E090637BF0906343E090637CF09063A2
:10007600767452F09062AE63A2019080A863A201EA
:100086007F06121C56020849906331E0C39408505B
:100096000302085290633EE0FF906377E06F6003CF
:1000A60002085290633FE0FF906378E06F600302BE
:1000B6000852906340E0FF906379E06F60030208A6
:1000C60052906341E0FF90637AE06F60030208524A
:1000D600906342E0FF90637BE06F600302085290FA
:1000E6006343E0FF90637CE06F6003020852906315
:1000F60076E0B444159062AEE0B4FF0E63A20190C0
:1001060080A863A2017F06121C5690668BE06003EE
:100116007401F090668C7464F09063767452F0907B
:100126006375E0646D60030202537BFF7A0E79DD2E
:100136001213597BFF7A0E79F790633EE0F52EA3F2
:10014600E0F52FA3E0F530A3E0F531A3E0F532A307
:10015600E0F533121359752EFF752F0F7530547550
:1001660031FF75320F7533607BFF7A0F792D1213CD
:10017600597BFF7A0F79691213597BFF7A0F79CF72
:100186001213597BFF7A0F79FC906344E0F52EA396
:10019600E0F52FA3E0F530A3E0F5311213597BFF0C
:1001A6007A10792690634DE0F52EA3E0F52FA3E0B3
:1001B600F530A3E0F5311213597BFF7A107954908C
:1001C6006351E0F52EA3E0F52FA3E0F530A3E0F5AB
:1001D600311213597BFF7A10798290633AE0F52E3B
:1001E600A3E0F52FA3E0F530A3E0F5311213597B18
:1001F600FF7A1079A5906336E0F52EA3E0F52FA3DC
:10020600E0F530A3E0F5311213597BFF7A1079C27D
:100216001213597BFF7A1079EBA20FE433F52E12F5
:1002260013597BFF7A11791B906681E0F52E121324
:10023600597BFF7A11794690668BE0F52E12135999
:100246001228417BFF7A117979121359229063752E
:10025600E0644C70737E117F7FFBFDFC122371906E
:10026600637DE0F526A3E0F527E4F529E52690630E
:100276007FF0A3E527F07E117FBA7C637D7F7B024A
:10028600122371E4F528852782852683E0FF747F93
:100296002528F582E43463F583EFF00527E527701A
:1002A6000205260528E528B410DC7E117FBD7C6397
:1002B6007D7F7B101223710529E529C3941040AC7C
:1002C6007E117FC012275922906375E0646C7060BE
:1002D600F52A7E117FC2FBFDFC122371E4F529E4A9
:1002E60090637FF0A3E52AF07E117FBA7C637D7F61
:1002F6007B02122371E4F528A82AE6FF747F2528DD
:10030600F582E43463F583EFF0052A0528E528B481
:1003160010E67E117FBD7C637D7F7B101223710505
:1003260029E529C3940840B77E117FC012275922B8
:10033600906375E0644B7061F52874672528F58233
:10034600E43463F583E0603274672528F582E4348B
:1003560063F583E0F4602374672528F582E434634B
:10036600F583E0FF747D2528F582E43463F583E0A8
:10037600B507100528E528B408C09061047432F06A
:100386000208499063757421F0300B030208497E18
:10039600117FFD122759020849906375E0B4521A7D
:1003A600200B077E127F051227599063757472F031
:1003B6007E637F757D08122FAB22906375E06449DA
:1003C6007045200B077E127F1012275990637DE03F
:1003D600F526A3E0F527E4F528852782852683E020
:1003E600FF747F2528F582E43463F583EFF0052753
:1003F600E527700205260528E528B480DC7E637FA4
:10040600757D8A122FAB22906375E0644370462097
:100416000B077E127F1812275990637DE0F526A3FD
:10042600E0F527E4F528852782852683E493FF7483
:100436007F2528F582E43463F583EFF00527E52769
:10044600700205260528E528B480DB7E637F757D6E
:100456008A122FAB22906375E0645A7053200B0703
:100466007E127F2112275990637DE0F526A3E0F5E1
:10047600277C637D7F7B80AF27AE261236A4E4F50A
:1004860028852782852683E493FF747F2528F582B5
:10049600E43463F583EFF00527E5277002052605AA
:1004A60028E528B480DB7E637F757D8A122FAB2218
:1004B600906375E06444600302054790637DE0FF46
:1004C60064447003020849EFB4310CC20B7E127FFC
:1004D6002D12275902084990637DE0B4300CD20BE7
:1004E6007E127F3912275902084990637DE0B432A3
:1004F6000CD20C7E127F4612275902084990637D62
:10050600E0B4330CC20C7E127F54122759020849FC
:1005160090637DE0B4340CD20D7E127F63122759AE
:1005260002084990637DE0B4350CC20D7E127F70DF
:1005360012275902084990637DE0FF12380E02081F
:1005460049906104E07013200B077E127F7E12270C
:10055600599063757421F00208499061047432F071
:10056600906375E0FFB45104C2AF80FEEF6457702C
:1005760045200B077E127F8C12275990637EE090F0
:100586006331F0E4F528906331E0FFE528C39F402E
:1005960003020849747F2528F582E43463F583E075
:1005A600FF90637DE0252824ADF582E43461F58370
:1005B600EFF0052880D0906375E06453600302066F
:1005C6006A200B077E127F9712275990633EE0FF41
:1005D6009061B6E06F703C90633FE0FF9061B7E0DA
:1005E6006F7030906340E0FF9061B8E0B5072490EB
:1005F6006341E0FF9061B9E0B50718906342E0FF00
:100606009061BAE0B5070C906343E0FF9061BBE0F0
:100616006F60169063757421F0300B030208497EF3
:10062600127FA6122759020849E4F528E4F549AFD6
:1006360028FE74AD2528F582E43461F583E0FD12C9
:1006460037000528E528C394FE40E1C2AFE4907F59
:10065600F0F0A3F0907FFD74AAF0A374FFF0A374EA
:1006660055F080FE906375E0644F704C90637DE0BA
:10067600F526A3E0F527E5274526700A200B077E19
:10068600127FAF122759200B077E127FB612275909
:10069600E4F528747F2528F582E43463F583E08544
:1006A6002782852683F00527E5277002052605287B
:1006B600E528B480DE020849906375E0FFB4452161
:1006C60090637DE0FDA3E0907FF0CDF0A3EDF0C256
:1006D600AF907FFD74AAF0A374FFF0A37455F08069
:1006E600FEEF6465600302085290637DE0FFA3E0BD
:1006F600907FF0CFF0A3EFF0E4F526F527D3907FB7
:10070600F1E09527907FF0E095264020E4F5492515
:1007160027FFE5263401FE852782852683E0FD1224
:1007260037000527E5277002052680D17E127FB89F
:100736001230B9EF4E6020120003906344EFF012BE
:100746000003906345EFF0120003906346EFF0124A
:100756000003906347EFF07E127FBE1230B9EF4E72
:10076600602012000390634DEFF012000390634E79
:10077600EFF012000390634FEFF012000390635006
:10078600EFF07E127FC41230B9EF4E6020120003E4
:10079600906351EFF0120003906352EFF0120003E2
:1007A600906353EFF0120003906354EFF07E127FD4
:1007B600CA1230B9EF4E602012000390633AEFF090
:1007C60012000390633BEFF012000390633CEFF0DE
:1007D60012000390633DEFF07E127FD01230B9EF26
:1007E6004E6020120003906336EFF0120003906310
:1007F60037EFF0120003906338EFF01200039063B6
:1008060039EFF0E4F528E4F549E5282401FFE4335F
:10081600FE74362528F582E43463F583E0FD12374D
:10082600000528E528C3944340DCC2AFE4907FF07E
:10083600F0A3F0907FFD74AAF0A374FFF0A37455A3
:0C084600F080FE7E637F757D08122FABF2
:010852002283
:10366C00AE07EEC39430400BEED394395005EE24E4
:10367C00D0FF22EEC39461400BEED394665005EE5E
:10368C0024A9FF22EEC39441400BEED3944650057F
:08369C00EE24C9FF22AF062253
:1037C2009062ADE004F070069062ACE004F09062AA
:0A37D200ACE0FEA3E0FF12376C220A
:100003001237C212366CEFC454F0FEC0061237C268
:0800130012366CD0E02FFF2231
:10351300E49069B5F01237C29069B6EFF0C3943006
:103523004018E0FFD3943950119069B5E02405F5B4
:1035330082E43461F583EFF080119069B5E02405EE
:10354300F582E43461F583E4F0800C9069B5E0041E
:10355300F0E0D3940840BE752900752A00752B004E
:0C356300E4F52C7B017A617905121D64EF
:01356F002239
:0430B9008E2B8F2C9F
:1030BD009062ACE4F0A374FFF01237C2EF606EF4CF
:1030CD00606B852C82852B83E493B507EC752D0100
:1030DD00E52C252DF582E4352BF583E493602590C1
:1030ED0062ADE0252DFF9062ACE03400FE12376C2E
:1030FD00E52C252DF582E4352BF583E493B50704F6
:10310D00052D80CCE52C252DF582E4352BF583E4BA
:10311D009370A6E52D24FFFFE434FFFE9062ADE031
:10312D002FF09062ACE03EF07E007F0122E4FEFFC6
:01313D00226F
:102AE3007E127FD61230B9EF4E70037F01227E1221
:102AF3007FD91230B9EF4E600C1237C2EF24D024C5
:102B0300FF920F8002D20F7E127FDF1230B9EF4E99
:102B1300600C1237C2EF24D0906681F08005E490F8
:102B23006681F07E127FE51230B9EF4E600C1237EA
:102B3300C2EF24D090668BF08005E490668BF07E24
:102B4300127FEB1230B9EF4E600C1237C2EF24D074
:102B530024FF92018002C20190633E63A20190664A
:102B63007B63A2017F06121C5630013B7E127FF16C
:102B73001230B9EF4E603012000390667BEFF01213
:102B8300000390667CEFF012000390667DEFF01275
:102B9300000390667EEFF012000390667FEFF01261
:0A2BA3000003906680EFF07F00222F
:10362500906576E0C3947C503D906576E0FE04F0AD
:1036350074B42EF582E43462F583EFF0BF0A279067
:103645006576E0FF04F074B42FF582E43462F58307
:10365500E4F0906576E0FF12313E9065767408F0EF
:073665009062B5E004F022C1
:1035CC009080007480F090633663A201F583F582DD
:1035DC0063A2017F08121C5690633E63A201908087
:1035EC008863A2017F0A121C56908092E4F0A374A7
:1035FC0032F0A37401F0906348E0FF9080B1F0903A
:10360C0080E1EFF09080957455F0A3F090800074F9
:09361C0001F090800974F0F02225
:1033BC00908009E04410F09080A0E0706C9080A1A7
:1033CC007482F09080A874FFF0A3F0A3F0A3F07FB8
:1033DC00039080AEEFF07FCBA3EFF07F039080AC37
:1033EC00EFF0A374CBF09080007402F09069A512FA
:1033FC0017F0000000009069A5E0908040F0906903
:10340C00A6E0908041F09069A7E0908042F090692E
:10341C00A8E0908043F0A3E4F0A3F0A3F0A3F09015
:09342C008018F0A3F0A3F0A3F056
:013435002274
:10357000908009E04440F09080D17482F07F039005
:1035800080DEEFF0A374CCF09080027402F09069BA
:10359000A91217F0000000009069A9E0908058F08F
:1035A0009069AAE0908059F09069ABE090805AF061
:1035B0009069ACE090805BF0A3E4F0A3F0A3F0A3EB
:0B35C000F0908030F0A3F0A3F0A3F027
:0135CB0022DD
:10343600908009E04420F09080B8E0706C9080B9EC
:103446007482F07F039080C6EFF07FCDA3EFF07F0C
:10345600039080C4EFF0A374CDF09080C074FFF0A9
:10346600A3F0A3F0A3F09080017402F09069AD126E
:1034760017F0000000009069ADE090804CF0906974
:10348600AEE090804DF09069AFE090804EF090698C
:10349600B0E090804FF0A3E4F0A3F0A3F0A3F09087
:0934A6008024F0A3F0A3F0A3F0D0
:0134AF0022FA
:1031C3008C268D27A907EAFDE975F018A424ACFF26
:1031D300E5F034808F82F583EDF0EBFDE975F018AF
:1031E300A4FFAEF024ACFBEE34808B82F583A3ED19
:1031F300F08527828C83E0FDEF24A8FFEE3480FE68
:103203008F82F583EDF08527828C83A3E08F828EF6
:1032130083A3F0852782852683A3A3E0FDE975F0C8
:1032230018A424A8FFE5F03480FE8F82F583A3A3BE
:10323300EDF08527828C83A3A3A3E08F828E83A3E3
:04324300A3A3F0222F
:062FAB008D2BAB07AA0606
:102FB100908000E030E5079065787401F022906917
:102FC100A5E0FCA3E0FDA3E0FEA3E0F52F8E2E8D8E
:102FD1002D8C2CAE02AF038E838F8263A201E52E6E
:102FE100540744C0F583852F8263A201AF2B121CC5
:102FF100C8E4FCFDFEE52F252BF52FEE352EF52E31
:10300100ED352DF52DEC352CF52C908040E52CF08F
:10301100A3E52DF0A3E52EF0A3E52FF09080007439
:1030210020F0AF2FAE2EAD2DAC2C9069A51217E478
:01303100227C
:063032008D26AB07AA0683
:10303800908002E030E5079065787403F02290698B
:10304800A9E0FCA3E0FDA3E0FEA3E0F52A8E298D0C
:10305800288C27AE02AF038E838F8263A201E529F5
:10306800540744D0F583852A8263A201AF26121C37
:10307800C8E4FCFDFEE52A2526F52AEE3529F529C2
:10308800ED3528F528EC3527F527908058E527F009
:10309800A3E528F0A3E529F0A3E52AF090800274BF
:1030A80020F0AF2AAE29AD28AC279069A91217E401
:0130B80022F5
:022DDF008F263D
:102DE100908001E030E5099065787402F07F00225F
:102DF1009069ADE0FCA3E0FDA3E0FEA3E0F52A8E1F
:102E0100298D288C2790667B63A201E5295407440C
:102E1100C8F583852A8263A2017F06121CDEE52A9A
:102E21002406F52AE43529F529E43528F528E43581
:102E310027F52790657963A201E529540744C8F570
:102E410083852A8263A201AF26121CDEE4FCFDFE0B
:102E5100E52A2526F52AEE3529F529ED3528F52827
:102E6100EC3527F52790804CE527F0A3E528F0A362
:102E7100E529F0A3E52AF09080017420F0AF2AAE95
:0D2E810029AD28AC279069AD1217E4AF26EB
:012E8E002221
:102478009081E0E0F5260526052605260526052691
:1024880005260526052605260526908010E0F5294F
:10249800A3E0F52AA3E0F52BA3E0F52C9081E1E079
:1024A800F5260526052605260526052605260526DC
:1024B800052605260526908014E0F52DA3E0F52EC7
:1024C800A3E0F52FA3E0F530E52FB52B08E530B5EF
:1024D8002C037F0022E4F526E52F540744E0F5831A
:1024E80085308263A20190637563A2017F08121D83
:1024F8000E90637763A2019062AE63A2017F061219
:102508001C56906375E0F527A3E0F528E4F52690BE
:102518006375E0702AA3E024F8F526E52F540744F4
:10252800E0F58385308274082582F582E43583F5E9
:102538008363A20190637563A201AF26121D0EAEDC
:1025480027E4FCFDE5302528F530E52F3EF52FED95
:10255800352EF52EEC352DF52D908014E52DF0A3B4
:10256800E52EF0A3E52FF0A3E530F090800074404D
:03257800F0AF269B
:01257B00223D
:101F08009081E6E0F5260526052605260526052600
:101F180005260526052605260526908028E0F529AC
:101F2800A3E0F52AA3E0F52BA3E0F52C9081E7E0E8
:101F3800F526052605260526052605260526052651
:101F480005260526052690802CE0F52DA3E0F52E24
:101F5800A3E0F52FA3E0F530E4F526E52FB52B0A2D
:101F6800E530B52C05C208022074E52F540744F06B
:101F7800F58385308263A20190637563A2017F08AF
:101F8800121D0E906375E0F527A3E0F528E52845B6
:101F98002770099080027410F07F0022906682E01A
:101FA800FFF46030906377E06F600302203B906637
:101FB80083E0FF906378E06F7079906684E0FF902B
:101FC8006379E06F706D906685E0FF90637AE06FEB
:101FD8006031805F906377E0906682F0906378E08C
:101FE800906683F0906379E0906684F090637AE07D
:101FF800906685F090637BE0FFA3E0906349CFF0A3
:10200800A3EFF0906375E0702AA3E024F8F526E5C5
:102018002F540744F0F58385308274082582F582B1
:10202800E43583F58363A20190637563A201AF264B
:10203800121D0EAE27E4FCFDE5302528F530E52F0E
:102048003EF52FED352EF52EEC352DF52DAF2CAEBA
:102058002BAD2AAC29AB30AA2FA92EA82DD3121745
:10206800D340099080027410F07F002290802CE504
:102078002DF0A3E52EF0A3E52FF0A3E530F0908036
:06208800027440F0AF26D7
:01208E00222F
:10220B009081E3E0F52605260526052605260526FD
:10221B000526052605260526052690801CE0F529B2
:10222B00A3E0F52AA3E0F52BA3E0F52C9081E4E0E5
:10223B00F52605260526052605260526052605264B
:10224B00052605260526908020E0F52DA3E0F52E2A
:10225B00A3E0F52FA3E0F530E4F526E52FB52B0A27
:10226B00E530B52C05C209022356E52F540744E887
:10227B00F58385308263A20190600463A2017F0E17
:10228B00121D24906004E0F527A3E0F52890600C64
:10229B00E0FFF4604590667BE0FEEF6E706EA3E0AE
:1022AB00FF90600DE06F706490667DE0FF90600EB4
:1022BB00E06F705890667EE0FF90600FE06F704C9F
:1022CB0090667FE0FF906010E06F7040906680E05A
:1022DB00FF906011E06F60048032D2D9906004E00F
:1022EB00702AA3E024F2F526E52F540744E8F58382
:1022FB00853082740E2582F582E43583F58363A2E3
:10230B000190600463A201AF26121D24AE27E4FCEA
:10231B00FDE5302528F530E52F3EF52FED352EF573
:10232B002EEC352DF52DAF2CAE2BAD2AAC29AB30C9
:10233B00AA2FA92EA82DD31217D35006E52845276F
:10234B0070099080017410F07F0022908020E52DA1
:10235B00F0A3E52EF0A3E52FF0A3E530F09080017C
:05236B007440F0AF26F4
:01237000224A
:042759008E2B8F2C08
:10275D00908000E030E5079065787401F022906973
:10276D00A5E0FCA3E0FDA3E0FEA3E0F5328E318DE4
:10277D00308C2FE532FFE5315407FEE42FF52EEEB8
:10278D0034C0F52D852E82F5837423F0052EE52EAC
:10279D007002052D532DC7F582852D83740AF00522
:1027AD002EE52E7002052D532DC790633E63A201B9
:1027BD00852D83852E8263A2017F06121CC87406A7
:1027CD00252EF52EE4352DF52D852B83852C826355
:1027DD00A201852D83852E8263A201121CACE4FC1F
:1027ED00FDFE9069A5E0F8A3E0F9A3E0FAA3E02FC0
:1027FD00FFEE3AFEED39FDEC38FCEF2408FFE43E28
:10280D00FEE43DFDE43CFC9069A51217E49069A53A
:10281D00E0908040F09069A6E0908041F09069A72B
:10282D00E0908042F09069A8E0908043F0908000A5
:03283D007420F014
:012840002275
:0A2371008E2B8F2C8C2D8D2E8B2FC0
:10237B00908000E030E5079065787401F022906959
:10238B00A5E0FCA3E0FDA3E0FEA3E0F5358E348DC4
:10239B00338C32E535FFE5345407FEE42FF531EE8F
:1023AB0034C0F530853182F5837423F00531E53186
:1023BB00700205305330C7F582853083740AF005FF
:1023CB0031E531700205305330C790633E63A20193
:1023DB0085308385318263A2017F06121CC8740687
:1023EB002531F531E43530F530852B83852C82632F
:1023FB00A20185308385318263A201121CAC8F361A
:10240B00EF2531F531E43530F530E52F6017852DAB
:10241B0083852E8263A20185308385318263A2017D
:10242B00AF2F121CC8E5362408252FF52FFFE4FC2F
:10243B00FDFEE5352FF535EE3534F534ED3533F559
:10244B0033EC3532F532908040E532F0A3E533F0D2
:10245B00A3E534F0A3E535F09080007420F0AF35A0
:0C246B00AE34AD33AC329069A51217E41A
:012477002242
:02313E008F3FC1
:10314000908000E030E5079065787401F022906986
:10315000A5E0FCA3E0FDA3E0FEA3E0F5438E428DD5
:10316000418C40E543FFE5425407FEE42FFFEE3477
:10317000C09062B463A201F5838F8263A201AF3F66
:10318000121CC8E4FCFDFEE543253FF543EE354245
:10319000F542ED3541F541EC3540F540908040E594
:1031A00040F0A3E541F0A3E542F0A3E543F09080B1
:1031B000007420F0AF43AE42AD41AC409069A5121F
:0231C00017E412
:0131C20022EA
:062926008E268F27AB0591
:10292C00908000E030E5079065787401F0229069A2
:10293C00A5E0FCA3E0FDA3E0FEA3E0F52D8E2C8D1D
:10294C002B8C2AE52DFFE52C5407FEE42FF529EE00
:10295C0034C0F528852982F5837423F00529E529EF
:10296C00700205285328C7F582852883EBF00529CA
:10297C00E5297002052890633E63A20185288385B2
:10298C00298263A2017F06121CC874062529F52929
:10299C00E43528F5285328C7E52685298285288320
:1029AC00F00529E529700205285328C7F5828528EA
:1029BC0083E527F00529E529700205285328C7E58A
:1029CC002D240AF52DE4352CF52CE4352BF52BE4D0
:1029DC00352AF52A908040E52AF0A3E52BF0A3E5F3
:1029EC002CF0A3E52DF09080007420F0AF2DAE2CD0
:0A29FC00AD2BAC2A9069A51217E478
:012A060022AD
:1034B000908009E04480F09080E97401F07F0990E9
:1034C00080F6EFF0A37464F09080037402F09080B3
:1034D00000E020E1F99068A11217F00000000090D0
:1034E00068A1E0908064F09068A2E0908065F09020
:1034F00068A3E0908066F09068A4E0908067F0A3F5
:10350000E4F0A3F0A3F0A3F090803CF0A3F0A3F0CC
:02351000A3F026
:013512002296
:102A07009081E9E0F52705270527052705270527ED
:102A170005270527052705270527908034E0F52892
:102A2700A3E0F529A3E0F52AA3E0F52B9081EAE0DE
:102A3700F52705270527052705270527052705273F
:102A4700052705270527908038E0F52CA3E0F52D0D
:102A5700A3E0F52EA3E0F52FE52EB52A08E52FB55F
:102A67002B037F0022AF2FAE2EAD2DAC2CAB2BAAA4
:102A77002AA929A828D31217D3400AAF2FAE2BEEC5
:102A87009FF527800AAF2FEFF404AE2B2EF527E52D
:102A97002E540744E0F583852F8263A2019068A531
:102AA70063A201AF27121D3CE4FCFDFEE52F25279D
:102AB700F52FEE352EF52EED352DF52DEC352CF5C4
:102AC7002C908038E52CF0A3E52DF0A3E52EF0A39C
:0B2AD700E52FF09080037440F0AF2763
:012AE20022D1
:02257C008F27A7
:10257E009080E8E0640660037FFF229068A1E0FC93
:10258E00A3E0FDA3E0FEA3E0F52B8E2A8D298C2877
:10259E00E4FFFEFDFCAB2BAA2AA929A828C312171B
:1025AE00D370609081F9E0F5289068A1E0FCA3E07B
:1025BE00FDA3E0FEA3E0FFE4FAF9F8EF2401FFEA41
:1025CE003EFEE93DFDE83CFC9068A11217E49068E0
:1025DE00A1E0FCA3E0FDA3E0FEA3E0FFE4F8EF24FE
:1025EE0001FFEA3EFEE93DFDE83CFC9068A11217B2
:1025FE00E4908064E0F528A3E0F529A3E0F52AA392
:10260E00E0F52B9068A563A201E52A540744D8F59E
:10261E0083852B8263A201AF27121CF6E4FCFDFE1C
:10262E00E52B2527F52BEE352AF52AED3529F5294B
:10263E00EC3528F528908064E528F0A3E529F0A371
:10264E00E52AF0A3E52BF09080037420F0AF2BAEBB
:0D265E002AAD29AC289068A11217E47F0076
:01266B00224C
:10376C00A2AF9219C2AF438E2075D2028F828E8384
:0C377C00E0FFE4F5D2538EDFA21992AFFB
:01378800221E
:10370000E5D220E0FBA2AF9219C2AF43D2028F8272
:103710008E83EDF075D25063D250A21992AFE5D2EC
:0337200020E0FBAB
:013723002283
:10324700E4FDED2401FFE433FE12376C74362DF5EF
:1032570082E43463F583EFF00DBD3FE6E4FDED2432
:103267007FFFE433FE12376C742D2DF582E4346151
:10327700F583EFF0742D2DF582E43461F583E0706A
:103287001B742D2DF582E43461F5837420F0742EC0
:103297002DF582E43461F583E4F080040DBD80BE32
:1032A700E49061ACF0FDEDFF7E0012376C74AD2D3C
:0D32B700F582E43461F583EFF00DBDFEE912
:0132C40022E7
:0236A4008B2B6E
:1036A600A2AF9219C2AF85A22C53A2FE8E838F823F
:1036B60005A28C838D827409121D52E52B53A2FE3E
:1036C60043A220121D5453A2DF852CA2A21992AF49
:0136D600FFF4
:0136D70022D0
:10378900A2AF9219C2AF8C838D82EF121D5243A250
:0C37990020121D5453A2DFA21992AFFFB2
:0137A5002201
:023724008F26EE
:10372600A2AF9219C2AFE4F5838D827406121D52C0
:10373600E52643A220121D5453A2DFA21992AF7FA1
:013746000181
:01374700225F
:023748008F26CA
:10374A00A2AF9219C2AFE4F5838D82740A121D5298
:10375A00E52643A220121D5453A2DFA21992AF7F7D
:01376A00015D
:01376B00223B
:101B7B00A907E7FFA805EF93C3966008403B74FCE9
:101B8B002FFF80F00F08EF93C3966008402B74FB78
:101B9B002FFF80E00F08EF93C3966008401B74FA89
:101BAB002FFF80D00F08EF93D3966008400B74F98A
:101BBB002FFF80C01F1F1F1F1FEF54FEF80303F7DB
:101BCB00E893FC08E893FD08E893FE08E893FF22EE
:101BDB0009E993C39D6008402974FB29F980F10939
:101BEB00E993C39E6008401A74FA29F980E209E967
:101BFB0093D39F6008400B74F929F980D3191919F5
:101C0B001919E9C313C313FF22740093F8ECC3989B
:101C1B004024701F740193F8EDC39840197014742D
:0E1C2B000293F8EEC398400E7009740393F80C
:101C3900EFC39840037F00227F0122EDF8E6F00808
:101C4900A3DFFA22EDF8E0F608A3DFFA22E0A363A6
:101C5900A201F0A363A201DFF475A2002263A2012D
:101C6900F0A363A20122E0A363A201F0A363A2018E
:101C7900E0A363A201F0A363A201E463A201F0A3BC
:101C890063A201DFE175A20022E0A363A2016DFE58
:101C9900936CFDEE058393FC158363A201DFEA755E
:101CA900A200227F00E493A363A201F00F600CA3BA
:101CB900E583C2E3F58363A20180EA75A20022E00D
:101CC900A363A201F0A3E583C2E3F58363A201DF65
:101CD900EE75A20022E0A363A201F0A3E583C2E4AA
:101CE900D2E3F58363A201DFEC75A20022E0A363CE
:101CF900A201F0A3E58344F8C2E5F58363A201DFFD
:101D0900EC75A20022E583C2E3F583E0A363A20197
:101D1900F0A363A201DFEE75A20022E583C2E4D23B
:0A1D2900E3F583E0A363A201F0A339
:101D330063A201DFEC75A20022E58344F8F583E09A
:101D4300A363A201F0A363A201DFEE75A20022F94F
:101D530022C002C004C00612FFF0D006D004D00295
:011D6300225D
:101919003E2A2C312CCFE0F0E0ECE5F2F0FB20E0A0
:10192900F1E8EDF5F0EEEDEDEEE3EE20EFEEF0F29D
:10193900E00A003E4C2C4930312C256C752CD1EA3B
:10194900EEF0EEF1F2FC20EEE1ECE5EDE02C3530C5
:101959002C3130302C3330302C3630302C31323081
:10196900302C323430302C343830302C3936303059
:101979002C31393230302C33383430302C3537363D
:1019890030302C3131353230300A003E422C49306A
:10199900322C2562752CCFF0EEE2E5F0FFF2FC2047
:1019A90043545320EFF0E820EFE5F0E5E4E0F7E5F4
:1019B9000A003E532C4931312C25752CC7E0E4E54A
:1019C900F0E6EAE020F1F2E0F0F2E020EFE5F0E500
:1019D900E4E0F7E82028ECF1290A003E4C2C4930D4
:1019E900342C25732CD0E5E6E8EC20EFE5F0E5E4AE
:1019F900E0F7E82C3820E1E8F22C3720E1E8F20A98
:101A0900003820E1E8F2003720E1E8F2003E4C2CF2
:101A19004931302C25732CCAEEEDF2F0EEEBFC20A7
:101A2900F7E5F2EDEEF1F2E82C302DCDE5F22C31AF
:101A39002DD7E5F2EDFBE920284556454E292C32F4
:101A49002DCDE5F7E5F2EDFBE920284F4444290ABD
:101A590000302DCDE5F200312DD7E5F2EDFBE9207F
:101A6900284556454E2900322DCDE5F7E5F2EDFB27
:101A7900E920284F444429003E532C4930372C256E
:101A890062752CC4EEF1F2E0E2EAE020EFF0E82022
:101A9900EFF0E8E5ECE5204E20E1E0E9F220283C12
:101AA900313236290A003E532C4930392C256275CA
:101AB9002CC4EEF1F2E0E2EAE020EFF0E820EFF0EA
:101AC900E8E5ECE520E1E0E9F2E02028302DEDE55C
:101AD900F220EAEEEDF2F0EEEBFF290A003C493084
:101AE900313D003C4930323D003C4930333D003CFA
:101AF9004931313D003C4930343D003C4930353DA8
:101B0900003C4930363D003C4931303D003C4930CC
:101B1900373D003C4930393D000AC1F3F4E5F02076
:101B2900E7E0EDFFF221000A2D3E000A4672616DE1
:101B390065206572726F722120000A3C2D00496E82
:101B490069745443500A004C697374656E54435068
:101B59000A00534F434B5F5443505F45535441422E
:101B69004C49534845440A000A2D3E20000A3C2DA1
:021B790020004A
:1037AC0052668D00000000000000000000000000C8
:0537BC00000000000008
:01380E002297
:03002300022BAD00
:0B2BAD00C0E0C083C082C0D075D0180B
:102BB800309841E50D25E9F5EB30D709E50C25F905
:102BC80004F5FB8006E50C25F9F5FBAF99D2917465
:102BD8009F2510F582E43466F583EFF00510E50EC5
:102BE8006005B51F02D2D9E510547FD3950840027D
:102BF800D2D9C298309965301260301707309704DF
:102C0800D2108056E512C3950F400AC212C290D264
:102C180018D2968045AF120512749F2FF582E434BE
:102C280067F583E0F51530151953157F3011282005
:102C3800D008201422631580801D30141A63158073
:102C48008015301112E5155215301406A2D0929B4A
:0C2C58008005A2D0B3929B851599C2990B
:092C6400D0D0D082D083D0E03240
:102841007BFF7A19791912135990689FE0FEA3E072
:10285100FFC3E49FFFE49EFEAB07FA3395E0F9F86E
:102861007F007E8C7D0A7C001217338F318E308D74
:102871002F8C2E7BFF7A19793C1213597BFF7A1921
:102881007994A217E433F52E121359AE09AF0A7CDD
:10289100007D0A1216538E2E8F2F7BFF7A1979BB7A
:1028A100121359201514752EFF752F1A75300A7BD6
:1028B100FF7A1979E41213598012752EFF752F1AB8
:1028C1007530107BFF7A1979E412135920111475B0
:1028D1002EFF752F1A75305A7BFF7A1A791612134B
:1028E100598029301414752EFF752F1A7530607BAD
:1028F100FF7A1A79161213598012752EFF752F1A45
:102901007530707BFF7A1A79161213597BFF7A1A88
:10291100798185082E1213597BFF7A1A79AF850EBA
:052921002E12135922E3
:10208F007E1A7FE61230B9EF4E600B12351390694E
:10209F00B11217E4800A9069B11217F00000258081
:1020AF009069B1E0F8A3E0F9A3E0FAA3E0FB7F00A9
:1020BF007E8C7D0A7C001217331217C590689FEE35
:1020CF00F0A3EFF0E47B0AFAF9F89069B1E0FCA312
:1020DF00E0FDA3E0FEA3E0FF121733A804A905AAB1
:1020EF0006AB07E47FB87E88FDFC1217338E0C8F8A
:1020FF000D7E1A7FEC1230B9EF4E600C1237C2EF23
:10210F0024D024FF92178002C2177E1A7FF212305A
:10211F00B9EF4E6012123513E47B64FAF9F8121618
:10212F00A88E098F0A8005E4F509F50A7E1A7FF853
:10213F001230B9EF4E6012123513E47B0AFAF9F838
:10214F001216A88E098F0A8005E4F509F50A7E1A82
:10215F007FFE1230B9EF4E600A1237C2EF24D0F56E
:10216F00158003751508E515B40704D2158002C252
:10217F00157E1B7F041230B9EF4E600C1237C2EF81
:10218F0024D024FF92118002C2117E1B7F0A1230CD
:10219F00B9EF4E600C1237C2EF24D024FF92148097
:1021AF0002C2147E1B7F101230B9EF4E600A123735
:1021BF00C2EF24D0F5158005E4F515C211E515B46D
:1021CF000104D211D214E515B40204D211C2147E47
:1021DF001B7F161230B9EF4E60071235138F088030
:1021EF00037508407E1B7F1C1230B9EF4E6007123B
:0B21FF0035138F0E8003E4F50E7F0007
:01220A0022B1
:1036D800C2A9438902758C48758A4875D90475DB77
:1036E8004875DC4875DD4875DE48E4F5E9F5F9C24A
:0836F800D9C2DAD28CD2DE2225
:10334100C212C218E4F512F50FF510C210D297D2CD
:103351009675130912208FC2ADE4F5C9D2CDD2CC36
:10336100C2C9C2CAF5CDF5CC90689FE0F5CBA3E008
:10337100F5CA85CBCD85CACCE4F59830110C201562
:10338100095387BFD29FD29E8002D29E438740C2FB
:103391009FC2ACC298C29975B81075B710D2CAD283
:1033A1009CD2AC1236D8C2D9E5E92464F5EB30D70A
:0B33B10006E5F904F5FB2285F9FB227C
:01380F002296
:102D2A00E4FF0F2405F582E43461F583E513F00F1F
:102D3A0074052401F582E43461F583E4F07C667D50
:102D4A0092FEED1DAA0470011CF5828A83E0FBAA9B
:102D5A00070F74052AF582E43461F583EBF00EBEA1
:102D6A0004E07C667D96E4FEED1DAA0470011CF564
:102D7A00828A83E0FBAA070F74052AF582E434618C
:102D8A00F583EBF00EBE04E07C667D9AE4FEED1D51
:102D9A00AA0470011CF5828A83E0FBAA070F740556
:102DAA002AF582E43461F583EBF00EBE04E07C661A
:102DBA007D9EE4FEED1DAA0470011CF5828A83E063
:102DCA00FBAA070F74052AF582E43461F583EBF058
:042DDA000EBE04E045
:012DDE0022D2
:05001E00D299D29022EE
:07380700D2CAD29CD2AC2210
:1032C5008F2620167630120B200B707E1B7F221264
:1032D500275922906378E0F513E52624FCFFF50FC6
:1032E5007D79758363058263A20190679F63A2015F
:1032F500121C56E4F512D212C296301702D210E50E
:103305000A4509601EC2DAE50A25E9F5EC30D70958
:10331500E50925F904F5FC8006E50925F9F5FCD252
:1033250013800312001E200B107E1B7F307C677DEF
:0C3335009FE52624FCFB122371C2182225
:102C6D0020D9037F0022C2D9E5E92410F5EB30D736
:102C7D0008E5F92428F5FB8006E5F92427F5FBE5A1
:102C8D0010547FD394005003022D27C291C2AF85FB
:102C9D001014631080531080D2AF30161DE51454FC
:102CAD0080249FF582E43466F58363A2019068A5C4
:102CBD0063A201AF14121C568058E4906475F0E5C0
:102CCD0014547FFFA3F090667AE0906477F0A3E54B
:102CDD0013F0E5145480249FF582E43466F5836384
:102CED00A20190647963A201121C56200B24309F1F
:102CFD00077E1B7F341227597E1B7F43E5145480BA
:102D0D00249FF582E43466AD82FCE514547FFB12FA
:0D2D1D002371C29FE514547FFF227F002226
:013810002295
:10266C003000489080E8E0700F1234B0300D077ED7
:10267C001B7F47122759C2169080E8E0B40E1290C7
:10268C0080037408F0300D077E1B7F50122759C24F
:10269C00169080E8E0B4060F20160C300D077E1B58
:1026AC007F5B122759D216C200050B30167420120C
:1026BC0007122A078F268003E4F526E526604730AB
:1026CC000D0C7E1B7F717C687DA5FB122371E5E9E7
:1026DC002410F5EB30D708E5F92428F5FB8006E546
:1026EC00F92427F5FB9068A563A20190679F63A26C
:1026FC0001AF26121C5685260FE4F512D290C2911A
:10270C00D212C296D299122C6D8F14E5146013124A
:10271C00257C300D0D7E1B7F767C687DA5AB14125D
:10272C002371301008209705C21012001E30130AB6
:10273C0030DA07C2DAC21312001E30120CE50BD3CA
:0C274C0094144008C212D21822E4F50BCD
:01275800225E
:0A37FD00201604122C6D227F00221A
:1037DC003016037F0022301805C2187F01227F00AB
:0137EC0022BA
:102F2B00020853E493A3F8E493A34003F68001F261
:102F3B0008DFF48029E493A3F85407240CC8C333A7
:102F4B00C4540F4420C8834004F456800146F6DF76
:102F5B00E4800B01020408102040809037A6E47E29
:102F6B00019360BCA3FF543F30E509541FFEE4936B
:102F7B00A360010ECF54C025E060A840B8E493A332
:102F8B00FAE493A3F8E493A3C8C582C8CAC583CA5D
:102F9B00F0A3C8C582C8CAC583CADFE9DEE780BE15
:0137C1000007
:10165300BC000BBE0029EF8DF084FFADF022E4CC7B
:10166300F875F008EF2FFFEE33FEEC33FCEE9DEC44
:10167300984005FCEE9DFE0FD5F0E9E4CEFD22ED8A
:10168300F8F5F0EE8420D21CFEADF075F008EF2FD4
:10169300FFED33FD4007985006D5F0F222C398FDC5
:0516A3000FD5F0EA2262
:1016A800E88FF0A4CC8BF0A42CFCE98EF0A42CFCE1
:1016B8008AF0EDA42CFCEA8EF0A4CDA8F08BF0A45F
:1016C8002DCC3825F0FDE98FF0A42CCD35F0FCEBBE
:1016D8008EF0A4FEA9F0EB8FF0A4CFC5F02ECD3983
:0F16E800FEE43CFCEAA42DCE35F0FDE43CFC22F0
:1016F70075F008758200EF2FFFEE33FECD33CDCCAA
:1017070033CCC58233C5829BED9AEC99E58298402C
:101717000CF582EE9BFEED9AFDEC99FC0FD5F0D609
:10172700E4CEFBE4CDFAE4CCF9A88222B800C1B933
:101737000059BA002DEC8BF084CFCECDFCE5F0CB71
:10174700F97818EF2FFFEE33FEED33FDEC33FCEBAA
:1017570033FB10D703994004EB99FB0FD8E5E4F965
:10176700FA227818EF2FFFEE33FEED33FDEC33FC52
:10177700C933C910D7059BE99A4007EC9BFCE99A46
:10178700F90FD8E0E4C9FAE4CCFB2275F010EF2F8B
:10179700FFEE33FEED33FDCC33CCC833C810D7078B
:1017A7009BEC9AE899400AED9BFDEC9AFCE899F8C6
:0E17B7000FD5F0DAE4CDFBE4CCFAE4C8F92259
:0E17C500C3E49FFFE49EFEE49DFDE49CFC2235
:1017D300EB9FF5F0EA9E42F0E99D42F0E89C45F06C
:0117E30022E3
:0C17E400ECF0A3EDF0A3EEF0A3EFF02278
:1017F000A8828583F0D083D08212180712180712AE
:101800001807121807E473E493A3C583C5F0C583D2
:10181000C8C582C8F0A3C583C5F0C583C8C582C842
:0118200022A5
:1012F700E53A242EF8E6053A22782B302002782E9C
:10130700E475F0011218790218212019EB7F2ED20B
:10131700198018EF540F2490D43440D4FF301D0B9C
:10132700EF24BFB41A0050032461FFE53B600215A8
:101337003B053EE53E7002053D30200D782BE475F8
:10134700F001121879EF0218670236257403D220CC
:101357008003E4C220F53A8B2B8A2C892DE4F53BD8
:10136700F53DF53EE53B60077F2012133280F575AA
:101377003CFFC21AC219C21BC21CC21EC21FC22115
:10138700121300FF700D3020057F00121343AF3E8C
:10139700AE3D22B4255FC2D5C21D121300FF24D073
:1013A700B40A00501A75F00A783B30D50508B6FF25
:1013B7000106C6A426F620D5047002D21C80D924C3
:1013C700CFB41A00EF5004C2E5D21D021543D21A5A
:1013D70080C6D21980C0D21B80BCD2D580BAD21E9B
:1013E70080B47F20121332201B077401B53B0040E5
:1013F700F11212F7FF12133202136BD221D21F80A0
:10140700951212F7FB1212F7FA1212F7F94A4B70FC
:101417000679147A167BFF201B2EE53B602A7E0097
:101427008E8275830012183A60060EEE653C70F0E6
:10143700C2D5EBC0E0EAC0E0E9C0E0EE12158AD001
:10144700E0F9D0E0FAD0E0FB121821FF60AAEBC068
:10145700E0EAC0E0E9C0E0121332D0E02401F9D09D
:10146700E03400FAD0E0FBE53C0460DCD53CD980F1
:10147700877BFF7A157986D21B809C791080027949
:1014870008C21FC2218008D2D5790A8004790AC20E
:10149700D5E53C047002F53CE4FAFDFEFF1212F7B5
:1014A700FC7B08201A131212F7FD7B1030190A1261
:1014B70012F7FE1212F7FF7B20EC3382D592D5503C
:1014C70013C3E43019069FFFE49EFEE4201A039D30
:1014D700FDE49CFCE4CBF8C21AEC700CCFCECDCC6B
:1014E700E824F8F870F38017C3EF33FFEE33FEED0F
:1014F70033FDEC33FCEB33FB994002FB0FD8E9EBF0
:10150700301A05F8D0E0C448B21AC0E00AEC4D4ED4
:101517004F78207B0070C2EAB53C0040BCC0E012A7
:10152700158CD0F0D0E0201A04C4C0E0C4B21AC0B1
:10153700F012131BD0F0D5F0EB02136B1218D8146E
:10154700085314825813D94C13D54214864F148E5E
:0F15570044148E4913EE431494551478461478B7
:101566004514784716345013DD2D13E12E14042B41
:1015760013E523140220161D2A139D48000013FCB0
:101586003F3F3F00790AA2D5201C14301E09B9102E
:10159600020404B9080104A2D5201F025001042048
:1015A6001B68921BB53B005034C0E07F20301C19ED
:1015B6007F30A21B721F721E500F1215E3C21BC290
:1015C6001FC21EC2217F30800F301E03E9C0E01209
:1015D6001332301E03D0E0F9D0E0B53BCC301E17F5
:1015E6007F30B9100C1213327F58301D077F788078
:1015F60003B90803121332301B057F2D0213327F05
:10160600202021F87F2B201FF322921B80CF286EEB
:10161600756C6C2900D21A1212F7301AF8C21A78B1
:101626003B30D50108F602139D2D5043495812123E
:10163600F72403B405004001E490162F93121323F8
:0D164600743A121323D21C753B0402148267
:101D64008B268A278928E4F532F531F530F52FF5ED
:101D74002DF52EE52A452B45296012EBC0E0EAC07B
:101D8400E0E9C0E0AB29AA2AA92B121889AB2605E1
:101D940028E528AA277002052714F9121821F5331B
:101DA400C394094007E533D3940D40E1E53364203F
:101DB40060DBE533B42D05432E038016E533B42BE5
:101DC40005432E01800C74FF2528F52874FF352760
:101DD400F527E52C60046410703FAB26AA27A928D8
:101DE40012182164306009E52C702E752C0A8029A4
:101DF40090000112183AFF64786004EFB45813435A
:101E04002E01752C1074022528F528E43527F527B2
:101E14008007E52C7003752C08AB260528E528AA55
:101E2400277002052714F9121821F533C394614071
:101E34000AE533D3947A50035333DF74D02533F552
:101E440033C3940A400CE5339411406D74F925337F
:101E5400F533E533D3952C5060432E018532378515
:101E64003136853035852F34AF2C7E00E4FCFDAB54
:101E740032AA31A930A82F1216A8C8ECC8C9EDC9D6
:101E8400CAEECACBEFCBE4FCFDFEEB2533F532EE14
:101E94003AF531ED39F530EC38F52FAF32AE31ADDE
:101EA40030FCAB37AA36A935A834D31217D3500364
:101EB400021E1D432E04021E1DE52E20E003E480B5
:101EC4002DE52A452B4529601EAB26E52824FFF97C
:101ED400E52734FFFAEBC0E0EAC0E0E9C0E0AB2953
:101EE400AA2AA92B121889E52E30E20774FFFFFEF7
:101EF400FDFC22E52EAF32AE31AD30AC2F30E10324
:041F04000217C522D9
:10182100BB010689828A83E0225002E722BBFE02C5
:09183100E32289828A83E49322F8
:10183A00BB010CE58229F582E5833AF583E0225063
:10184A0006E92582F8E622BBFE06E92582F8E222AD
:0D185A00E58229F582E5833AF583E49322C7
:10186700BB010689828A83F0225002F722BBFE0160
:02187700F3225A
:10187900FAE6FB0808E6F925F0F618E6CA3AF62270
:10188900BB011A89828A83D0F0D0E0F8D0E0F9D080
:10189900E0FAD0E0FBE8C0E0C0F00219075016E911
:1018A900F8D083D082D0E0F9D0E0FAD0E0FBC08252
:1018B900C0830218FEBBFE16E9F8D083D082D0E0BF
:0F18C900F9D0E0FAD0E0FBC082C08302191022F0
:1018D800D083D082F8E4937012740193700DA3A39F
:1018E80093F8740193F5828883E4737402936860B3
:0618F800EFA3A3A380DFB3
:0918FE00EBF608EAF608E9F6220F
:09190700EBF0A3EAF0A3E9F022E1
:09191000EBF208EAF208E9F22208
:00000001FF
